:020000040000FA
:06000000703002303A28C6
:08000800A000030EA100831209
:1000100081018B100B11210E8300A00E200E090010
:0C007400203084008001840A6030040207
:10008000031C3C281230B00039218316FF23900056
:10009000831283160C308505870183128501870141
:1000A000073099000030831691009F008312C830FA
:1000B00083168100831231309000003083168C004B
:1000C000831210308B00831600309B001C141A081A
:1000D0008312BC00831610309B001C141A08831274
:1000E000BD00762181018E018F010B118B100B1049
:1000F0008C018B178E20311990201D21B30B8C2879
:10010000031085190314B90DF030390203197F214A
:100110000F30390203197B2183217A2864000800FB
:10012000080031110130B7008B13203037078316D8
:100130009B001C141A088312A40010303707831682
:100140009B001C141A088312A30000303707831683
:100150009B001C141A088312A2008B17321CB628AD
:1001600022090339A200A309A409A5090130370215
:10017000031DBF283D18BF283D143E144F210130F8
:100180003702031DC8283D1CC8283D103E147321AA
:10019000C928B70A02303702031808009428013032
:1001A000B600B300B400B500B70085018701B113F4
:1001B0008E20B30BF528031085190314B90DF03008
:1001C000390203191329B41F8501B41F8701B40B29
:1001D000F5283708B6080319B6000319F328FF30CD
:1001E00085008700B6039630B400311DD828311140
:1001F000321CFF282D090339AD00AE09AF098B135E
:1002000020303707BB002F08BA00262110303707EF
:10021000BB002E08BA00262100303707BB002D088E
:10022000BA0026218B1785018701B70AB601023073
:100230003702031CD828762108003E1C08003E1017
:100240001030BB003D08BA00262108008B133A0885
:1002500083161C159A003B089B0055309D00AA3060
:100260009D009C1464009C1832291C1183128B176A
:100270000800831620309B001C141A088312DF002C
:10028000FF30D5000230D6000C30D700BA30D8008D
:100290003730D900DA30DA006F30DB000800013087
:1002A000BD000430C200C5000530C400C600CA004D
:1002B0000730C100C300C700C800C9005F19C117DB
:1002C0005F19C2175F19C317DF19C4175F1AC51763
:1002D0005F1AC6175F1AC7175F1AC8175F1BC917BF
:1002E000DF18CA170800850187010800BD013D1409
:1002F0003D184F2108003D143E144F2108003D10C9
:100300003E147321080001303D05031908005F19F0
:100310008B295C1805165F198F29DC1885165F1963
:1003200093295C190514DF199729DC1985145F1AC4
:100330009B295C1A87145F1A9F29DC1A07155F1A1C
:10034000A3295C1B07145F1AA729DC1B87165F1BF8
:10035000AB295D180716DF18AF29DD188715E630C1
:100360000E02031CC7295F1D05165F1D85165F1D44
:100370000514DF1D85145F1E87145F1E07155F1EA1
:1003800007145F1E87165F1F0716DF1C87158F086F
:10039000031908008F01850187015508DE00C52378
:1003A000D5005608DE00C523D6005708DE00551CD0
:1003B000C523D7005808DE00D51CC523D80059082E
:1003C000DE00551DC523D9005A08DE00D51DC52302
:1003D000DA005B08DE00551EC523DB005F1D0A2A1C
:1003E000C11B052AC11C0512C11CF9290512581987
:1003F0000516CB0B1B2A5608CB00C101D51BC11417
:10040000D81BC1105818C1101B2A0512CB0B1B2A70
:10041000C1031B2AC1080319051603191B2ACB0B9C
:100420001B2AD51BC1035508CB00D5185C14D51E5B
:100430005C10D51D5C105F1D372AC21B322AC21CFE
:100440008512C21C262A851258188516CC0B482AFC
:100450005608CC00C201D61BC2145A18C210D619B5
:10046000C210482A8512CC0B482AC203482AC20867
:10047000031985160319482ACC0B482AD61BC20338
:100480005608CC00D61ADC14561DDC10561FDC10A2
:100490005F1D642AC31B5F2AC31C0510C31C532A9B
:1004A00005105A190514CD0B752A5708CD00C30144
:1004B000D71BC314D51AC310D719C310752A05103A
:1004C000CD0B752AC303752AC30803190514031934
:1004D000752ACD0B752AD71BC3035708CD00571AB1
:1004E0005C15571F5C11D71D5C11DF1D912AC41BC1
:1004F0008C2AC41C8510C41C802A8510D51B851429
:10050000CE0BAD2A5808CE00C401D81BC414D71A8C
:10051000C410D819C410AD2A8510CE0BAD2AC4035F
:10052000AD2ADF1F9C2ACE0BAD2A5808CE00D51B62
:10053000DC15DA1FDC11AD2AC40803198514031970
:10054000AD2ACE0BAD2AD81BC4035808CE00581ACA
:10055000DC15D81FDC11D81DDC115F1EC92AC51B94
:10056000C42AC51C8710C51CB82A8710D51A871441
:10057000CF0BDA2A5908CF00C501D91BC514561A6A
:10058000C510D81BC510DA2A8710CF0BDA2AC5038D
:10059000DA2AC508031987140319DA2ACF0BDA2AD5
:1005A000D91BC5035908CF00D91B5C16D91F5C1293
:1005B000D91C5C125F1EF62AC61BF12AC61C071145
:1005C000C61CE52A0711D71A0715D00B072B5A08A6
:1005D000D000C601DA1BC614D51AC610D619C6102B
:1005E000072B0711D00B072BC603072BC6080319CF
:1005F00007150319072BD00B072BDA1BC6035A0864
:10060000D0005A1ADC165A1EDC12DA1FDC125F1EEA
:10061000232BC71B1E2BC71C0710C71C122B071030
:1006200059190714D10B342B5B08D100C701DB1B10
:10063000C714D719C710DB19C710342B0710D10BFB
:10064000342BC703342BC708031907140319342BA1
:10065000D10B342BDB1BC7035B08D100DB195C1704
:10066000DB1D5C135B1E5C135F1E502BC81B4B2BEA
:10067000C81C8712C81C3F2B871258198716D20B2B
:10068000612B5608D200C801D91BC8145A19C810CA
:10069000551AC810612B8712D20B612BC803612B2E
:1006A000C808031987160319612BD20B612BD71BBE
:1006B000C8035908D200561ADC17561EDC13DA1F7D
:1006C000DC135F1F7D2BC91B782BC91C0712C91CAB
:1006D0006C2B071255190716D30B972B5808D3000C
:1006E000C901D61BC914D91AC910D819C910972B1A
:1006F0000712D30B972BC903972B5F1C882BD30BA7
:10070000972B5708D300D61B5D14D81F5D10972B6D
:10071000C908031907160319972BD30B972BD51A62
:10072000C9035808D300D61B5D14D81F5D10DF1C09
:10073000B32BCA1BAE2BCA1C8711CA1CA22B871154
:10074000D51B8715D40B08005508D400CA01D51B4A
:10075000CA14561ACA10D619CA1008008711D40B29
:100760000800CA030800CA080319871503190800FE
:10077000D40B0800D81BCA035608D400591ADD143C
:10078000591EDD10DA1FDD100800C001DE08031954
:10079000DE035E184014DE1A40144008C0015E1CDF
:0E07A0004014DE1E4014C005C00C5E0C0800A4
:084000000D000300040008009C
:02400E00CC01E3
:10420000FF00FF00FF00FF00FF00FF00FF00FF00B6
:10421000FF00FF00FF00FF00FF00FF00FF00FF00A6
:104220000100FF00FF00FF00FF00FF00FF00FF0094
:10423000FF00FF00FF00FF00FF00FF00FF00FF0086
:104240000300FF00FF00FF00FF00FF00FF00FF0072
:10425000FF00FF00FF00FF00FF00FF00FF00050060
:10426000FF00FF00FF00FF00FF00FF00FF00FF0056
:10427000FF00FF00FF00FF00FF00FF00FF00FF0046
:10428000FF00FF00FF00FF00FF00FF00FF00FF0036
:10429000FF00FF00FF00FF00FF00FF00FF00FF0026
:1042A000FF00FF00FF00FF00FF00FF00FF00FF0016
:1042B000FF00FF00FF00FF00FF00FF00FF00FF0006
:1042C000FF00FF00FF00FF00FF00FF00FF00FF00F6
:1042D000FF00FF00FF00FF00FF00FF00FF00FF00E6
:1042E000FF00FF00FF00FF00FF00FF00FF00FF00D6
:1042F000FF00FF00FF00FF00FF00FF00FF000000C5
:00000001FF
